:030000000219FDE5
:03000B000200AA46
:03002B0002015679
:03005B000202E8B6
:030073000202D5B1
:1000800002030406080C10182030406080040608A3
:100090000C10182030406080A0C00003070F1F0D17
:1000A0000D04050D050205030302C2AFC0D0C0E078
:1000B000206214E5256009E473E525F4F58AD2622F
:1000C000D0E0D0D0D2AF3285268AC262E526F46075
:1000D00029D0E0D0D0C292C291C290D2AF32C292A7
:1000E000C291C290206F0C2066097405D5E0FDE531
:1000F0007B4290D0E0D0D0D2AF32758A00C28DD290
:100100006201F301B9306805206602D29201B9306C
:100110006805206602D29101B9306805206602D2D6
:100120009001B9C29530680A2066077446D5E0FD93
:10013000D29201B9C29430680A2066077446D5E0AD
:10014000FDD29101B9C29330680A2066077446D582
:10015000E0FDD29001B9C2AFC2AD53E6EFC0D0C04E
:10016000E0D2D3D2AFC2CEE52A6007207449152A67
:1001700021B77800790020742EE580307E01F430BC
:10018000E70278FF53DACF207E0343DA20307E0384
:1001900043DA10C2D8C271E580307E01F430E70244
:1001A00079FFC3E89970CB306103752A1820740376
:1001B000752A18885CD27020740DE52B6004152B0D
:1001C00021C743DA01C2D82070024136A85C206101
:1001D00002C2702074367982B70431C3E894F040CB
:1001E0000374F0F8E8C4540F28F87984B703024187
:1001F0000CC313C3138721200802C313200A06C3AC
:10020000C898F8410C28F8500374FFF88822E52DAF
:1002100054066022206B1FE536C333C333F8E56410
:10022000C313C313F9C3952240028922E82522F59E
:100230002250037522FF7882B6044E852224A8241A
:10024000C3E52495614002A861C3E895634002A814
:10025000638825E56670024187C3E8AA669A500361
:10026000E8FAE4F9EAC333FBE568F45B29400D25BD
:1002700067F8E56760021567400B41870AC3E567C9
:100280009A5002056778FF8826C3E525944040020E
:10029000D26420CF0AD0E0D0D043E610D2AD32C233
:1002A000CF053A7801E52A6005307402152AC3E5C6
:1002B0005C94014005755F0041CB75600075690075
:1002C000E55F2401F55F5003755FFFD0E0D0D043B8
:1002D000E610D2AD32C2AF53E67F7592FA7593FF46
:1002E000C260759104D2AF32C2AF53E6EFC2ADC067
:1002F000D0C0E0C0F0D2D3D2AFA8FBA9FCC2D830A6
:100300007102614F53DACF207E0343DA10307E034F
:1003100043DA20D271E580307E01F420E7026126C5
:1003200088278928A17C53DACF207E0343DA203046
:100330007E0343DA10C2D8C271307402A16878001B
:10034000E580307E01F430E702A168885CA150535B
:10035000DACF207E0343DA20307E0343DA10C27105
:10036000206102812853DACF207E0343DA10307EE9
:100370000343DA20C2D8D27188578958C3E895550B
:10038000F8E99556F97B007E087A00C3E8948CE979
:1003900094005005755B00811A882178A2E6A82197
:1003A0006055C3E894C8E994005008E4D2E4FB7AAD
:1003B0000A61F5C3E89468E994015008E4D2E3FBCC
:1003C0007A0F61F5C3E894D0E994025008E4D2E2D0
:1003D000FB7A1E61F5C3E894A0E994055008E4D2C5
:1003E000E1FB7A3C61F5C3E89498E994085008E48D
:1003F000D2E0FB7A787E00C3E89559FCE9955AFD76
:1004000030E70AECF42401FCEDF43400FD755B00E8
:10041000C3EC9AED9E5003755B018859895A855744
:10042000558558567802A150C3E89527F8E99528D4
:10043000F9307C02A134307B02A134307A02A12D44
:10044000207502814BE9FDE8FC816AE9C313F9E8F4
:1004500013F8307902A12DE9C313F9E813F83078C5
:1004600002A12DE9C313FDE813FC20612CC3EC9419
:0F0470001CED940240028181ED701EC3EC94C814
:10047F0050180529E52970021529C3E529940A505A
:10048F0002A168755C00D270A168E5296002152988
:10049F007888E6F97400207F087896B90302789E71
:1004AF00E624FAFEE43400FFC3EC9EFCED9FFD92C0
:1004BF0008B90310A2085007207609D27681D330ED
:1004CF007602C276A2085016B9030DECF42401FC93
:1004DF00EDF43400FD0204ED78007900A134B90386
:1004EF0015EC33FCED33FDC3EC940AFCED9400FDE9
:1004FF0050047C007D00C3EC94FFED94004006781F
:10050F00FF7900A134EC8572F0A4C5F0A2F733F89F
:10051F007900400302055078FF7900020550E9C3C6
:10052F0013F9E813F8307C0EE9600278FFC3E81383
:10053F0038F8E43400F9C3E894FFE99400400278F6
:10054F00FF885CD270206102A168741FF4552F4B95
:10055F00F52FC274EB7002D274752A1830740375BC
:10056F002A0A306102A17C20740353DAFE2074033F
:10057F00752B06D0F0D0E0D0D0D2AD43E610327953
:10058F00010205AC79030205AC790A0205AC791EAC
:10059F000205AC79640205AC79C80205AC7817E4A2
:1005AF00D5E0FDD8FAD9F6227A147B780205D37AF2
:1005BF00107B8C0205D37A0D7BB40205D37A0B7BAB
:1005CF00C80205D37902E4C294D5E0FDD291D5E0FB
:1005DF00FDC291D5E0FDD294D5E0FDE920E002D235
:1005EF009230E002D290E573D5E0FDE920E002C23F
:1005FF009230E002C2907496D5E0FDD9C9EAF8D5E1
:10060F00E0FDD8FBDBBEC29422C37C007D0075F0F9
:10061F000005F0EA33FAEB33FB50F6EB13FBEA136A
:10062F00FAC3E9FFE8FEE89AF8E99BF95004EFF9FD
:10063F00EEF8B3EC33FCED33FDD5F0DFEDF9ECF86C
:10064F0022E889F08A20D2D4F8A9F07B0030F70B8A
:10065F007BFFF42401F8E9F43400F9E88520F0A4D5
:10066F00ADF0F8E98520F0A4AFF0FEED2EF974009F
:10067F003FFA7C04C3EA13FAE913F9E813F8DCF440
:10068F008BF030F70AE8F42401F8E9F43400F9E8C4
:10069F0089F0C2D4F8A9F0227882B60403020702C7
:1006AF00C3E55C940140030206CC852224E4F544A3
:1006BF00F545F546F547F548C26E0207027882E622
:1006CF00FCD26EE522F523783879C7AA40AB41C337
:1006DF00EB13FBEA13FAEC146013C3EB13FBEA13EF
:1006EF00FAEC14146007C3EB13FBEA13FAD1188862
:1006FF0044894522C3E5449523F8E5459400F95014
:10070F000CC3E89480E994FF4016020733C3E894C2
:10071F007FE994005003020733787F790002073393
:10072F00788079FF8849894A22E5492546F8E54AC4
:10073F003547F9854A20E4300701F43548FA30E7A8
:10074F0009C3EA94F04015020771C3EA940F5003EE
:10075F0002077178FF79FF7A0F020771780079002D
:10076F007AF0C3E5249561500AC374019524500BA8
:10077F0002078FE54A20E70E02078FE54A30E706AA
:10078F00884689478A482278A5E6FAC3E54933F8AF
:10079F00E54A33F9D150E930E70BC3E89480E99487
:1007AF00FF4013E1C9C3E8947FE994005002E1C907
:1007BF00787F7900E1C9788079FFE820E715C3E5F4
:1007CF002398F84009C3E8940140030207F0780129
:1007DF000207F0E8F424012523F840030207F0781C
:1007EF00FF884B2278A6E6FAA847A948D150E930EE
:1007FF00E70CC3E89401E994FF4016020824C3E80C
:10080F0094FFE99400500302082478FF790002084E
:10081F0024780179FFE920E715C3E54B98F84009E3
:10082F00C3E89401400302084B780102084BE8F437
:10083F002401254BF8400302084B78FF88242278C7
:10084F00FFC26420693D206A12D264C3E541940A55
:10085F004009C3E52594405002C26479A1E76023A3
:0D086F00E541601F74FF8541F0848539F07C
:10087C00306A0375F005A4F8C5F0600278FFC3E890
:10088C0095645002A864886322C3E5409440E54116
:10089C009401E56350031401A6046002F56322027F
:1008AC0008AE2275E890227883E6FFE5E820ECF7A5
:1008BC00A8BDA9BE0570C3E57094084052757000C0
:1008CC00E9FA79A0E76044EA7007E571601B020859
:1008DC00E9C3E895716010E5715006600C140208CC
:1008EC00F50460F90208F5E571F571C3946D401BD0
:1008FC007561C0C394044013756180C39404400BAC
:10090C00756140C39404400375610075BB0622E514
:10091C00612410500274FFF5617982B70402214200
:10092C00C3A861E524985002A824C3E8956340024B
:10093C00A86388258826E570B4070375BB1022745C
:10094C003279A787F0A4C5F0A2F733F8C3E8956114
:10095C004002A8618822882488258826886422750C
:10096C0040007541F022C2AF75C820A8CCA9CDAA11
:10097C003A30CF010A75C824D2AFAB3BAC3C883BB4
:10098C00893CC3E89BF8E99C206908F9306702416F
:10099C007E21DBAD3D8A3DF9EA9DFA600478FF7952
:1009AC00FFAE3EAF3F8B3E8C3FA83BA93CC3E89EBD
:1009BC00F8E99FF9C3E54113FBE54013FAE82AF582
:1009CC0040E93BF54150067540FF7541FF4125AAB2
:1009DC0040AB41AC40AD417E047F02C3EB9404407C
:1009EC00021E1FC3EB940840021E1FC3ED13FDEC47
:1009FC0013FCDEF7C3EA9CFAEB9DFBEF6009C3E93D
:100A0C0013F9E813F8DFF7EA28FAEB39FB8A408B85
:100A1C004150067BFF8B408B41C3EB94025002D2BA
:100A2C00673069047F0341507892E6FFC3E5379441
:100A3C008240110FC3E53794A040010FC3EF940619
:100A4C0040027F057E02E541C4540FF9E541C454D0
:100A5C00F0F8E540C4540F28F8C3E89EFAE9940076
:100A6C00FB4009C3EA9402EB940050047A02E4FBC5
:100A7C0041CAAA40AB41EBC4FEEAC4540F4EFCC3BE
:100A8C00EA9CFAEB9400FBC3E813C313F8EA28FAC8
:100A9C00EB3400FB8A408B41C3EB94024002C267EB
:100AAC007802EBC4FE7B00EAC4540F4EFAC3EA98FA
:100ABC00FA4005C3940250027A027892E6FF306045
:100ACC000241CA855192855293D26043E680C3E4B9
:100ADC009AF8E49BF93067026156E8FAE9FBD3E92E
:100AEC0013FDE813FC88518952C3EF94036038EF6F
:100AFC0020E00DE82CF8E93DF9ECFAEDFB020B1FB8
:100B0C00E828F8E939F9C3E82402F8E93400F97A5D
:100B1C00FE7BFFC3EF9403400E8A538B54884D89A0
:100B2C004E8C4F8D50618A885389548A4D8B4E8CD4
:100B3C004F8D503069127553F07554FF754FF07529
:100B4C0050FF7551F07552FF618AE8FAD3E813FC37
:100B5C008851C3EF94036020EF20E007E82CF8ECF9
:100B6C00FA6176E8282402F87AFEC3EF9403400871
:100B7C008A53884D8C4F618A88538A4D8C4FE56817
:100B8C00C3335002646BF5683060026194753402B3
:100B9C00D26043E680E52D54066034A840A941C3D9
:100BAC00E913F9E813F8C3E913F9E813F830690409
:100BBC00E92440F9C2AF53E67F759100C3E498F580
:100BCC0094E499F595759104D26043E680D2AF22F6
:100BDC00D265754300752000306C03752040020B04
:100BEC00FBD265754300752040306C03752000788E
:100BFC00017901206720E52D54066002C265791445
:100C0C00E541C313700104F8C39414400278143006
:100C1C006904781B791B206010E543600C30690374
:100C2C00D53404D26D819E719C0543E59BF45440F0
:100C3C00B52002818830690908C3E8994001188100
:100C4C002220650A08C3E899400261FB8122C26533
:100C5C00C2AF53E67F75910030671275940075959D
:0F0C6C00FE759104D26043E680D2AF61FBAE40CB
:100C7B00AF41C3E49EF594E49FF595816DC3E533D5
:100C8B009401500261FB30650261FBD802819C81AB
:100C9B0022C26DC2AF53E67F759100855394855484
:100CAB0095759104854D92854E93D26043E680D223
:100CBB00AFE52D54066008206A020533020CDA30CA
:100CCB006D0D206C0A2065071581158102155D22BB
:100CDB0078003064053065027801E53775F007A4BC
:100CEB00F9E5F028F5F0E9A2F013A2F113A2F21343
:100CFB00F537C394785003753778C3E5379538408B
:100D0B0008D266C292C291C290306002A114854F84
:100D1B0092855093D26043E68022207D16C2AF7538
:100D2B004202C294D295306202D290D2AF759F111B
:100D3B00020F14C2AF754202C294D293306202D238
:100D4B0092D2AF759F11020F14307243207D20C2D7
:100D5B00AF754203900134757B10C290C293306221
:100D6B0004D291A172D294D2AF759F01020F14C21B
:100D7B00AF754203900134757B10C292C2953062FD
:100D8B0004D291A192D294D2AF759F21020F14205D
:100D9B007D17C2AF75420390010FC290306202D231
:100DAB0091D2AF759F01020F14C2AF754203900130
:100DBB000FC292306202D291D2AF759F21020F14F3
:100DCB00207D16C2AF754204C295D293306202D217
:100DDB0091D2AF759F21020F14C2AF754204C2931B
:100DEB00D295306202D291D2AF759F01020F1430AF
:100DFB007243207D20C2AF754205900123757B2085
:100E0B00C291C294306204D292C118D295D2AF75FE
:100E1B009F11020F14C2AF754205900145757B08F7
:100E2B00C291C294306204D290C138D293D2AF75C2
:100E3B009F11020F14207D17C2AF7542059001055B
:100E4B00C291306202D292D2AF759F11020F14C2BF
:100E5B00AF754205900119C2913062EBD290D2AFBF
:100E6B00759F11020F14207D16C2AF754206C293F7
:100E7B00D294306202D292D2AF759F01020F14C28C
:100E8B00AF754206C295D294306202D290D2AF7542
:100E9B009F21020F14307243207D20C2AF75420197
:100EAB00900145757B08C292C295306204D290C105
:100EBB00BED293D2AF759F21020F14C2AF75420100
:100ECB00900123757B20C290C293306204D292C1F1
:100EDB00DED295D2AF759F01020F14207D17C2AFE2
:100EEB00754201900119C292306202D290D2AF7555
:100EFB009F21020F14C2AF754201900105C29030C1
:100F0B006202D292D2AF759F01C266229001037525
:100F1B007B00C292C291C290C295C294C293C2622C
:100F2B0022788076090876090876040876FF087619
:100F3B00030876FF08760B08760108760108760120
:100F4B00788C76010876FF0876FF0876FF0876FF27
:100F5B000876FF0876030876FF0876FF0876FF0809
:100F6B0076250876D0087628087650087604087619
:100F7B00FF08760208760008767A0876FF08760175
:100F8B00087601087600087603087600227887E653
:100F9B00FFC2727888E6C394036008C27DE630E135
:100FAB0002D27DC27E7889E630E102D27EC3EF9415
:100FBB00026008758E01D273020FCB758E00C2735F
:100FCB00227880E6149000809378A5F67881E61459
:100FDB009000809378A6F67886E61490008D93782F
:100FEB00A7F67886E6F539C3940250037539027873
:100FFB009CE67538FFB402037538A0B4030375384B
:10100B008278A3E61490009A93F566120F172222AA
:10101B007896E6FA7897E6FB7888E6B40305C3EB97
:10102B00940EFB307F047A007BFFC3EB9AFCC394D6
:10103B008250027C827572000572EC8572F0A4C33B
:10104B00E5F0947D40F222D27F111B12059D7A00B0
:10105B007B007C10120593E55C2AFA74003BFBDCE9
:0F106B00F37C04C3EB13FBEA13FADCF7FEC27F3E
:10107A00111B22E5EF20E6037520000520903FFFB3
:10108A00E520146006901DFF146000930460037548
:10109A00EF1053D9BF7581C043FF8012058E75EFDB
:1010AA000043B203E5B3240220E70DF521E5E3206E
:1010BA00E0068521B343E301120F177580FF75A47B
:1010CA000075F19075D47F75900075A53F75F23F54
:1010DA0075D50075A60175E241120F17E4F8F6D826
:1010EA00FD756801120F2C1215AE7898867375304B
:1010FA0001C2AF1205A71205B712059D1205BE124D
:10110A00059D1205C512059DC2AF78FA79FA308796
:10111A0007D9FBD8F7021C00120F98120FCC111A2C
:10112A00111B78988673120F1775881075890275C6
:10113A00C82475910475D84075A82275B80275E659
:10114A0090759B80759D0075D10E75BC5875BB0650
:10115A0075BA1175E88012058ED2AF1208AB7536D2
:10116A000053DACF207E0343DA20307E0343DA10BD
:10117A0043DA01C2D8C2711205A7D2617B037A0C85
:10118A00E55B70077A0CDB0302111212059D2070D1
:10119A0003021112C270E55CC3940240E1E52F54C8
:1011AA001F855E5DF55EB55DD5DAD5C26153DACFCE
:1011BA00207E0343DA20307E0343DA10C2D8C2719C
:1011CA0078A2E67008D274E52F54E0F52FC275753F
:1011DA0029001205A2307409C3E529940A4002D2F3
:1011EA007512059378023074027800C3E55C984062
:1011FA00F0C2AF1205B71205B71205B7D2AF120582
:10120A00A7754C007888E6B4030241EA1205937880
:10121A008CE6C3940150030212EAE530C3940150EC
:10122A00030212EA207435C3E55C94FF50030212EC
:10123A00EAC2AF1205CCD2AF1205A2C3E55C940193
:10124A0050EFC2AF1205B71205981205B7D2AF1206
:10125A0005A2C3E55C94FF40E90217567F02D27FDC
:10126A00111B1205A2C2AFC27F111BAE5CC3E55CA3
:10127A00947FD2AF407412058EC2AF1205CCD2AFA2
:10128A00DFDC1152C3EE7897F61205A71215F01299
:10129A0016D97F0AD27F111B1205A2C2AFC27F11D3
:1012AA001BAE5CC3E55C947FD2AF50E612058EC2DA
:1012BA00AF1205B71205981205B7D2AFDFD6115291
:1012CA00EE24037896F61205A71215F012170812E3
:1012DA0005A2111BC3E55C94FF5002412E0217566A
:1012EA00C3E55C954C4003855C4C1205A2780179F4
:1012FA0088E7B403027805C3E55C984002410EC250
:10130A00AF1205CC1205CC1205CCD2AF1205A775C7
:10131A003000E4F531F5320531E531F4703F05323C
:10132A00789AE67819146012783214600D787D1470
:10133A00600878FA146003753200C3E53298401DDC
:10134A00120F1712058E153275310078998673C2FD
:10135A00AF1205CCD2AF789886731205A2120598FF
:10136A00E52A700530740221127801207402780689
:10137A00C3E55C9840A17888E6C39403600312052C
:10138A00A2E52A7003021112C2AF120F17E4F52266
:10139A00F523F524F525F526F567D2AF7885E6C35A
:1013AA0033F565E4F544F545F546F547F548F57036
:1013BA00F52CF52DF53775700875BB1012058E12D0
:1013CA0008AFE5E820ECFBA8BDA9BEE97001F888E2
:1013DA00711208B375700875BB10120F98C2AF75F9
:1013EA0061FF12094B852261852262852263D2AF91
:1013FA0075220175240175250175260185606975B7
:10140A006A017888E6B40307C27D307602D27DD2BB
:10141A0068D269753300120E71120EA012096B128E
:10142A00097212096B12097212096B120BED12067C
:10143A00A7120CDB120D25120972120BDC306E0397
:10144A0012070320670312084E3067031208951229
:10145A000CDB120D54120972120BED306E031207D7
:0D146A0038120CDB120DCB120972120BDCD4
:10147700306E03120796120CDB120DFA1209721264
:101487000BED306E031207F3120CDB120E7112090B
:10149700721208AF120BDC120CDB120EA01208B38B
:1014A7001209723069328564618564628560697585
:1014B7006A0179187A0CC3E53399400FC269D26A79
:1014C7008A358564618564630214DFC3E55C940132
:1014D7004003021435021565306A1D206C1AE53584
:1014E700147006C26AD26B8135F535C3E55C940189
:1014F700400302143502156575360078FA79A4E7BA
:1015070060027803C3E55F985054307404E52A609D
:101517004D7888E6B40317207D05207607A135307E
:101527007602A135206C07D26C856461817478F0EE
:10153700306C058564617820C3E541985002813598
:10154700306C1BC26CC27D307602D27DD26A753593
:101557001285646181350536E55C6002A1687536E0
:1015670000C2AF120F177887E6FE7602120F98783F
:1015770087EEF6E4F522F523F524F525F526F5653E
:10158700752C00752D00D2AF1205A2120F1778A483
:10159700E66006D292D291D290307409C3E53694B0
:1015A7000440022112611C901A0D7820121632E5B0
:1015B70020B4550CA3121632E520B4AA030215D0A5
:1015C700120F2C1215F00215EF901A0378807B0A80
:1015D700121632A308DBF9901A0F788C7B191216B2
:1015E70032A308DBF9901A2822C2AF12167112161D
:1015F7004B901A00740E121637A37406121637A3EF
:101607007415121637901A0378807B0A121636A3C0
:1016170008DBF9901A0F788C7B19121636A308DBB2
:10162700F9121684121662901A2822E493F622E61B
:10163700438F01538FFD75EF0275B7A575B7F1F0AD
:10164700538FFE22438F02438F0175EF0275B7A5B3
:1016570075B7F1901A0DF0538FFC22901A0D74553F
:10166700D137901A0E74AAD137227A3079D07820E0
:10167700901A40D132E520F709A3DAF7227A3079B8
:10168700D0901A40E7D13709A3DAF922AB74A875CD
:10169700BB01027980BB02027981BB03027982BB5D
:1016A70004027984BB05027986BB06027992BB07DF
:1016B700027987BB080279A3BB0902799CBB0A029E
:1016C7007988BB0B027989E8F7227C051205A7DC2C
:1016D700FB22C2AF1205B71205BE1205C51205CC13
:1016E7001205981205B71205BE1205C51205CC12D0
:1016F70005981205B71205BE1205C51205CCD2AF63
:1017070022C2AF1205CC1205C51205BE1205B712CB
:1017170005981205CC1205C51205BE1205B71205AC
:10172700981205CC1205C51205BE1205B7D2AF2215
:10173700AE74AF75C2AF1205B71205B71205B7126F
:101747000598DEF21205CC120598DFF8D2AF22D148
:10175700D9D1D1D1D1757401757501757600F1377D
:101767007C05AD5C1205A7C3ED955C70F5C3E55C20
:101777009401400AC3E55C94FF4032021792D1936B
:10178700B1F0D1D9C2AF75EF10D1D1DCD50576C391
:10179700E5769403500280C6D1D10575E57414909F
:1017A700009F93F808C3E57598500280AED1D1D158
:1017B700D10574C3E574940C5002809C120F2CB1B0
:0817C700F0C2AF75EF10D1D1A3
:0319FD0002107D58
:101A00000E0615090904FF03FF0B01010155AA0188
:101A1000FFFFFFFFFF03FFFFFF25D0285004FF0259
:091A2000007AFF0101000300FF40
:101A400023585031324123202020202020202020E4
:101A500023424C48454C4923463333302320202031
:101A60002020202020202020202020202020202076
:101C0000C2AFC2D353D9BF7581C043B20343FF8073
:101C1000752438752503B1C975EF0275E24043F1AB
:101C20008053A47F75D4FFD2877DFA780379E67C50
:101C300010752200752300901DD67B0675249875BB
:101C400025013087028142208708D8FBD9F9DCF7CB
:101C500081B4308708D8FBD9F9DCF781B4B189E4C5
:101C600093A3C39A6004DDC381B4DBDBB17B600264
:101C7000812B7B08E493FAA3B15CDBF87A30B15C8A
:101C8000752200752300B17BEAFCEBFDC3ED94FEE9
:101C9000400EB17B8A278B28ED30E0048A828B834B
:101CA000B17B7AC270D8C3ED94FE601350CEBD00F4
:101CB00025EC60097520007521FF0200008100A855
:101CC00027A9280809D804D90281D3B17FEA89AAB3
:101CD000F281C50D81A0C3ED94035049EDA2E092BD
:101CE000007AC5C3E5829400E583941C50902000DF
:101CF00010438F02438F0175B7A575B7F1F030001F
:101D00001FA827A9280809438F01538FFDD804D99C
:101D100002A12089AAE275B7A575B7F1F0A3A10DBC
:101D2000538FFC817C7AC1BD030CE493A3FAB140CC
:101D3000DCF8B138817C817EAA22AB23B15CEBFA5E
:101D4000EA6222752608C3E52313F523E52213F57D
:101D50002250066323A0632201D526EAB1C9B1C986
:101D600075260AEAF4200102D287300102C287B147
:101D7000C9C3134002C201D526EB22B17FEAFB2082
:101D80008702A17F308702A184752608AE24AF2583
:101D9000C3EF13FFEE13FEB1CDB1C9C3EA13308711
:101DA000024480FA30E703632201C3E52313F523DD
:101DB000E52213F52250066323A0632201D526D91C
:101DC000E52265236523F52222AE24AF250E0FDE22
:101DD000FEDFFCD20122424C48656C693437316326
:041DE000F3300601D5
:00000001FF
